:100000000C9484000C94A3000C94A3000C94A30003
:100010000C94A3000C94A3000C9499010C94A300DD
:100020000C94A3000C94A3000C94A3000C94A300C4
:100030000C94A3000C94A3000C94A3000C94A300B4
:100040000C94A3000C94A3000C94A3000C94A300A4
:100050000C94190A0C94A3000C94A3000C94A30014
:100060000C94A3000C947A110C94B3060C94A30086
:100070000C94A3000C94A3000C94A3000C94A30074
:100080000C94A3000C94A3000C94A3000C94850A78
:100090000C94D1120C946F060C94A3000C94A30042
:1000A0000C94A3000C94A3000C9420010C94A300C6
:1000B0000C94A3000C94A3000C94A3000C94A30034
:1000C0000C94A3000C94A3000C94A300494E464941
:1000D0004E4954594E414ECDCCCC3D0AD7233C1706
:1000E000B7D13877CC2B329595E6241FB14F0A0053
:1000F0000020410000C84200401C4620BCBE4CCA43
:100100001B0E5AAEC59D740011241FBECFEFD1E265
:10011000DEBFCDBF1DE0A0E0B2E0ECEFFEE400E00A
:100120000BBF02C007900D92AA32B107D9F710E1B8
:10013000AAE2BDE001C01D92A13EB107E1F70E9415
:10014000551D0C947C270C9400008A3010F4809389
:100150002F0E089510922B0E10922C0E10922D0E31
:1001600010922E0E089510922B0E10922C0E1092BB
:100170002D0E10922E0E10922F0E1092300E4FEF69
:1001800040936D0E30E130936E0E21E020936F0EA0
:1001900088E998E09093710E8093700E1092720E21
:1001A0004093730E3093740E2093750E9093770ED8
:1001B0008093760E3093780E2093310E1092320E8B
:1001C00010927C0E80E090E0FC01EE0FFF1FED5CD2
:1001D000F14F11821082019688309105A9F780E0D5
:1001E00090E0FC01E55DF14F808F0196883091052C
:1001F000C1F780E090E024E6FC01E55DF14F20A32B
:10020000019688309105C1F78FEF9FE39093640EBC
:100210008093630E9093660E8093650E88E08093C2
:10022000670E8FEF9FE19093690E8093680E8CE2CA
:1002300091E090936B0E80936A0E10926C0E08956D
:100240001F920F920FB60F920BB60F9211242F939D
:100250003F934F935F936F937F938F939F93AF934E
:10026000BF93EF93FF931092A5001092A4002091EA
:10027000220230912302E091300E8091A10DF0E036
:1002800044E0EE0FFF1F4A95E1F7E80FF11DEC5D2A
:10029000FD4F8081280F311D3093A9002093A800C5
:1002A00080912E0D863034F08FEF90E09093A9006E
:1002B0008093A800A8950E9420110E94FA03E09163
:1002C0002F0E8091A10DF0E034E0EE0FFF1F3A9564
:1002D000E1F7E80FF11DEC53FD4F81E060810E94D2
:1002E000110480E293E00197F1F780912E0D8F5F6A
:1002F00080932E0D86E00E948B048F7180932F0DCA
:1003000060912E0D4091A10D0E942211FF91EF915D
:10031000BF91AF919F918F917F916F915F914F911D
:100320003F912F910F900BBE0F900FBE0F901F901B
:1003300018951F920F920FB60F920BB60F921124C1
:10034000EF920F932F933F934F935F936F937F930E
:100350008F939F93AF93BF93EF93FF93DF93CF93CD
:1003600000D0CDB7DEB719821A828FE00E948B04CD
:10037000A89582FF07C086E00E948B048F7180934E
:100380009E0D2AC183FF28C180919F0D9091A00DE1
:10039000019709F002C181E39DE06CE6AE014E5F7A
:1003A0005F4F9E012F5F3F4F0E940C05882309F489
:1003B00013C18981882309F40FC120912B0E30913C
:1003C0002C0E40912D0E50912E0E8091310D90915A
:1003D000320DA091330DB091340D82179307A4070D
:1003E000B50709F088C08091A4009091A500909372
:1003F0002D0D80932C0D1092A5001092A4008091D9
:100400002E0D882331F48CE390E0909323028093A7
:1004100022028091220290912302E091300E2091DD
:10042000A10D0A96F0E0B4E0EE0FFF1FBA95E1F7D8
:10043000E20FF11DEC5DFD4F2081820F911D909325
:10044000A9008093A800A8950E941E1100912E0D6E
:10045000E090A10D81E39DE060919E0D40919D0D86
:100460002A810E94E113082F86E00E948B048F717D
:1004700080939D0D8430F8F40023E9F0E0912F0E75
:100480008091A10DF0E0A4E0EE0FFF1FAA95E1F727
:10049000E80FF11DEC53FD4F82E060810E941104D2
:1004A00080E293E00197F1F781E39DE0602F70E037
:1004B0000E94080419C00E94FA03E0912F0E809157
:1004C000A10DF0E074E0EE0FFF1F7A95E1F7E80F61
:1004D000F11DEC53FD4F81E060810E94110480E228
:1004E00093E00197F1F7A89580912E0D8093300D40
:1004F00010922E0D71C080912B0E90912C0EA09118
:100500002D0EB0912E0E0097A105B10509F064C023
:1005100080919E0D853008F45FC0A8950E941E1141
:1005200080912B0E90912C0EA0912D0EB0912E0E3D
:100530002091310D3091320D4091330D5091340D99
:1005400082179307A407B50771F08091350D81508C
:10055000823048F420932B0E30932C0E40932D0EB6
:1005600050932E0EA8950E94FA03E0912F0E8091D1
:10057000A10DF0E064E0EE0FFF1F6A95E1F7E80FD0
:10058000F11DEC53FD4F81E060810E94110480E277
:1005900093E00197F1F7A8951FC00E94FA03E0913C
:1005A0002F0E8091A10DF0E054E0EE0FFF1F5A9541
:1005B000E1F7E80FF11DEC53FD4F81E060810E94EF
:1005C000110480E293E00197F1F7A89586E00E947C
:1005D0008B048F7180939D0D0F900F90CF91DF91C1
:1005E000FF91EF91BF91AF919F918F917F916F910B
:1005F0005F914F913F912F910F91EF900F900BBE14
:100600000F900FBE0F901F901895DF93CF9300D0DF
:1006100000D0CDB7DEB789E492E0A0E0B0E08983F6
:100620009A83AB83BC83CE01019660E070E044E026
:1006300050E00E946E258BE29EE064E070E042E5AF
:1006400050E00E946E250F900F900F900F90CF9169
:10065000DF910895EF92FF920F93DF93CF93CDB781
:10066000DEB768970FB6F894DEBF0FBECDBF198214
:100670001A821B821C820E94B300CE01019660E0A8
:1006800070E044E050E00E945E2589819A81AB8150
:10069000BC8105E0E02EF12CEC0EFD1E8954924049
:1006A000A040B040D1F48BE29EE064E070E042E50F
:1006B00050E00E945E2580E092E00E946A0820914E
:1006C0002B0E30912C0E40912D0E50912E0EC70105
:1006D000B90140E020E001E018C080E192E00E9412
:1006E0006A0869817A81C70140E020E001E00E9448
:1006F000F706C7010E946A0880E292E00E946A0839
:10070000C70169E472E040E020E00E94F706C701FB
:100710000E946A088DE092E00E946A0868960FB60F
:10072000F894DEBF0FBECDBFCF91DF910F91FF9048
:10073000EF9008958AEF90E0909323028093220235
:100740000E942A0380912F0E8A3010F480932F0E7E
:100750000E9436040E94FA03E0912F0E8091A10DB1
:10076000F0E094E0EE0FFF1F9A95E1F7E80FF11D1E
:10077000EC53FD4F81E060810E94110485E06FE041
:1007800040E020E00E94AF040E94D5031092A50033
:100790001092A40080912202909123029093A900CC
:1007A0008093A8000E941E1108951092A500109237
:1007B000A4001092A00085E08093A1008FEF90E04C
:1007C0009093A9008093A800E2E7F0E08081826026
:1007D00080837894089594B7977F94BFE0E6F0E023
:1007E00090819861908387708860808384B7877FC9
:1007F00084BF08958091A10D8F3030F48091A10DB8
:100800008F5F8093A10D02C01092A10D80E008952A
:100810009C01862FB9010E9464052C9A2C9880E0D7
:1008200008951F93182F262F88E06FE140E00E9463
:10083000AF04812F90E09093A00D80939F0D113015
:1008400019F482E066E008C085E060E847E021E056
:100850000E94AF0482E069E00E947C048EE06CE0BC
:100860000E947C04789480E01F9108950F931F9359
:1008700084E00E9457040CEF13E0C8010197F1F7E0
:1008800017982C988CE090E00197F1F7179A82E086
:1008900068E00E947C04C8010197F1F781E06FE1F4
:1008A00040E00E949C0480E01F910F9108950F9AF0
:1008B000249A95B1936095B994B1976094B92398AF
:1008C00090E59CBD9CB59C7F9CBD9DB59E7F9DBDCC
:1008D0002CB5982F9370922B9CBD9DB586958695CF
:1008E0008170982B9DBDEAE6F0E080818C6080836A
:1008F00080E28CBBED9A0895806C9FB7F89428989D
:100900008EBD0DB407FEFDCF6EBD0DB407FEFDCF4D
:10091000289A9FBF08958F7380689FB7F89428988E
:100920008EBD0DB407FEFDCF8EBD0DB407FEFDCF0D
:100930008EB5289A9FBF0895FF920F931F93062F9D
:10094000F42E0E948B04082310E002C01595079531
:10095000FA94E2F7802F1F910F91FF900895DF9294
:10096000EF92FF920F931F93D82EF62EE42E022FB4
:100970000E948B046F2D6095682310E002C0000F69
:10098000111FEA94E2F7F0226F298D2D0E947C045A
:100990001F910F91FF90EF90DF900895CB01089584
:1009A000FC01DA015FB7F894289880E28EBD0DB49F
:1009B00007FEFDCF1EBC0DB407FEFDCF4EB564177C
:1009C00030F1942F20E030E01EBC0DB407FEFDCFC7
:1009D0008EB52827022E2295207F2025032E322F28
:1009E00022952F700226269532272327220F220FC9
:1009F000220F20258083915011F03196E5CF10977A
:100A000039F01C92232B21F481E08C9301C04068C3
:100A1000289A5FBF842F0895FF920F931F93CF935F
:100A2000DF938C01EA01D901FFB6F894289880E29F
:100A30008EBD0DB407FEFDCF1EBC0DB407FEFDCF6D
:100A40009EB5691708F436C020E030E040E050E081
:100A5000692F70E01CC01EBC0DB407FEFDCF8EB523
:100A6000F801E20FF31F80834827042E4295407F50
:100A70004025052E542F42954F7004264695542745
:100A80004527440F440F440F40252F5F3F4F261743
:100A9000370708F3109729F01C92452B11F481E0D9
:100AA0008C93209741F01EBC0DB407FEFDCF8EB590
:100AB000888301C09068289AFFBE892FDF91CF916B
:100AC0001F910F91FF900895982FFB012FB7F89475
:100AD000289880E68EBD0DB407FEFDCF9EBD0DB4F7
:100AE00007FEFDCF80818EBD915011F03196F7CF7A
:100AF0000DB407FEFDCF289A2FBF0895FC01DA013F
:100B00003FB7F894289880E28EBD0DB407FEFDCF64
:100B10001EBC0DB407FEFDCF2EB56217A0F0922FBC
:100B20001EBC0DB407FEFDCF8EB58083915011F031
:100B30003196F6CF109741F01EBC0DB407FEFDCFE5
:100B40008EB58C9301C02068289A3FBF822F0895EC
:100B5000833309F080E0089583E30895E82FF0E0FF
:100B6000EE0FFF1FED57F14F20813181C90108952C
:100B7000E82FF0E0EE0FFF1FED57F14F11821082CA
:100B800008959B01AC01529A53985A9A5B9A64E07B
:100B9000220F331F441F551F6A95D1F760E072E1A1
:100BA0008AE790E00E94AE24215030401092CD00A0
:100BB0002093CC0080E48093C80088E98093C9002A
:100BC00086E08093CA00789408959B01AC01689AEE
:100BD0006998709A719A74E0220F331F441F551F51
:100BE0007A95D1F760E072E18AE790E00E94AE2446
:100BF000215030401092C5002093C40080E48093BF
:100C0000C00088E98093C10086E08093C200789498
:100C10000895FC018091800E8823D1F4F093820E18
:100C2000E093810E6093800E2091850E3091860EA8
:100C3000808190E0822793279093860E8093850E83
:100C400080818093CE008091C90080628093C9002A
:100C50008091800E8823E1F70895FC0180917D0E3C
:100C60008823D1F4F0937F0EE0937E0E60937D0E87
:100C70002091830E3091840E808190E0822793270B
:100C80009093840E8093830E80818093C600809120
:100C9000C10080628093C10080917D0E8823E1F7BE
:100CA0000895DF93CF930F92CDB7DEB78983CE013E
:100CB000019661E00E942D060F90CF91DF9108957B
:100CC000DF93CF930F92CDB7DEB78983CE01019624
:100CD00061E00E9409060F90CF91DF9108951F9265
:100CE0000F920FB60F920BB60F9211242F933F93D2
:100CF0008F939F93EF93FF93E091810EF091820E7B
:100D00003196F093820EE093810E31978091800EA0
:100D100081508093800E8091800E882391F0809185
:100D2000850E9091860E2181332727FD3095282747
:100D300039273093860E2093850E81818093CE00D3
:100D400005C08091C9008F7D8093C900FF91EF910C
:100D50009F918F913F912F910F900BBE0F900FBEDF
:100D60000F901F9018951F920F920FB60F920BB60F
:100D70000F9211242F933F938F939F93EF93FF93A1
:100D8000E0917E0EF0917F0E3196F0937F0EE0930E
:100D90007E0E319780917D0E815080937D0E8091E3
:100DA0007D0E882391F08091830E9091840E218195
:100DB000332727FD3095282739273093840E209339
:100DC000830E81818093C60005C08091C1008F7D14
:100DD0008093C100FF91EF919F918F913F912F914F
:100DE0000F900BBE0F900FBE0F901F901895BF92E3
:100DF000CF92DF92EF92FF920F931F93DF93CF93E7
:100E0000CDB7DEB72C970FB6F894DEBF0FBECDBFBF
:100E10006C01FB01B42EE22E77FD02C0FF2408C056
:100E2000F095E195FF4F8DE2D6018C93FF24F3946A
:100E300040E08E010F5F1F4F10C0200F311FCF0108
:100E40006AE070E00E949B24805DD9018C93CF0101
:100E50006AE070E00E949B24FB01242F30E04F5F8A
:100E6000EA30F10554F7020F131F8E2F805DF80151
:100E70008083642FCE01019620E305C0FC01E60FBC
:100E8000F11D20836F5FE616C8F76B15B8F3862F48
:100E900090E09E012F5F3F4FF901E80FF91F10828C
:100EA0000197D901A80FB91F019640E050E08C01CD
:100EB0002E2D30E07EE214C0C801841B950B8217F2
:100EC000930729F4F601EF0DF11D7083F394F601F9
:100ED000EF0DF11D8C918083F3944F5F5F4F11975D
:100EE000461750F3F601EF0DF11D1082C6012C9646
:100EF0000FB6F894DEBF0FBECDBFCF91DF911F912B
:100F00000F91FF90EF90DF90CF90BF9008954F9298
:100F10005F926F927F928F929F92AF92BF92CF9289
:100F2000DF92EF92FF920F931F93DF93CF93CDB792
:100F3000DEB72C970FB6F894DEBF0FBECDBF3C01D5
:100F40006A017B01422E502E77FD02C099240DC00C
:100F5000F094E094D094C094C11CD11CE11CF11C0D
:100F60008DE2F30180839924939488245E01089490
:100F7000A11CB11C19C00A0D1B1DC701B6012AE036
:100F800030E040E050E00E94D024605DF8016083D2
:100F9000C701B6012AE030E040E050E00E94D024D2
:100FA000C901DA016C017D01082D10E08394FAE09B
:100FB000CF16D104E104F104F4F6A00EB11E8C2D7D
:100FC000805DF5018083482DCE01019620E305C0A8
:100FD000FC01E40FF11D20834F5F5416C8F7441540
:100FE000B8F3842F90E09E012F5F3F4FF901E80F87
:100FF000F91F10820197D901A80FB91F019620E0AF
:1010000030E0BC01052D10E05EE214C0CB01821B74
:10101000930B8017910729F4F301E90DF11D50831B
:101020009394F301E90DF11D8C91808393942F5FCC
:101030003F4F1197241750F3F301E90DF11D108272
:10104000C3012C960FB6F894DEBF0FBECDBFCF9173
:10105000DF911F910F91FF90EF90DF90CF90BF90A5
:10106000AF909F908F907F906F905F904F9008957A
:10107000DC010D900020E9F71197A81BB90B6A2F2E
:101080000E942D060895EF92FF920F93DF93CF9366
:10109000CDB7DEB72A970FB6F894DEBF0FBECDBF2F
:1010A000BC017E010894E11CF11CC70140E020E076
:1010B00001E00E94F706C7010E9438082A960FB681
:1010C000F894DEBF0FBECDBFCF91DF910F91FF909F
:1010D000EF900895DC010D900020E9F71197A81B0F
:1010E000B90B6A2F0E9409060895CF92DF92EF9202
:1010F0000F93DF93CF93CDB7DEB72A970FB6F8944F
:10110000DEBF0FBECDBFAB01BC016E010894C11C98
:10111000D11CC60120E000E0EE24E3940E94870782
:10112000C6010E946A082A960FB6F894DEBF0FBE69
:10113000CDBFCF91DF910F91EF90DF90CF900895C9
:10114000EF92FF920F93DF93CF93CDB7DEB72A973D
:101150000FB6F894DEBF0FBECDBFBC017E01089470
:10116000E11CF11CC70140E020E001E00E94F7060D
:10117000C7010E946A082A960FB6F894DEBF0FBE18
:10118000CDBFCF91DF910F91FF90EF9008958098A0
:1011900081988298839886E880937A0080E480938F
:1011A0007C000895806480937C0086E880937A00B8
:1011B00080917A00806480937A0080917A0084FF25
:1011C000FCCF2091780030917900C9010895609199
:1011D000700E7091710E660F771F660F771F40912A
:1011E000A30D80916E0E481798F48091720EE42F33
:1011F000F0E0E80FF11DEE0FFF1FE957F14F80817E
:10120000918162E070E00E949B246059784E0CC08E
:1012100080916F0E823061F480916E0E90E0242FE9
:1012200030E08217930724F04F5F4093A30D02C074
:101230001092A30DCB0108956091760E7091770EF8
:10124000660F771F660F771F4091A20D8091740E75
:10125000481798F48091780EE42FF0E0E80FF11D24
:10126000EE0FFF1FE957F14F8081918162E070E03E
:101270000E949B246059784E0CC08091750E82307C
:1012800061F48091740E90E0242F30E08217930770
:1012900024F04F5F4093A20D02C01092A20DCB012B
:1012A000089510928500109284001092950010927B
:1012B0009400089590916D0EE82FF0E0EC59FC4FEA
:1012C000E0819E1709F44FC08091730E8E1709F4C8
:1012D0004AC0E23029F1E33030F4EE2349F0E13046
:1012E00009F041C011C0E33039F1E430E1F530C01C
:1012F000CB0162E070E00E949B246059784E7093AD
:101300008900609388000895CB0162E070E00E943C
:101310009B246059784E70938B0060938A000895E7
:10132000CB0162E070E00E949B246059784E70937C
:101330008D0060938C000895CB0162E070E00E9404
:101340009B246059784E709399006093980008959B
:10135000CB0162E070E00E949B246059784E70934C
:101360009B0060939A000895CF93DF93259A269A65
:10137000279AE0E8F0E01082A1E8B0E01C9226E8AD
:1013800030E0E901198218828081826080838C912B
:1013900080618C938081886A80838C9181608C933A
:1013A00060E070EF7983688320E737E1309389004C
:1013B0002093880030938B0020938A0030938D0017
:1013C00020938C00EFE6F0E08081816080836C9A4E
:1013D0006B9AE0E9F0E01082A1E9B0E01C9246E9E6
:1013E00050E0EA01198218828081826080838C91AA
:1013F00080618C938081886A80838C9181608C93DA
:1014000079836883309399002093980030939B00F0
:1014100020939A0088EE9DEF90939500809394001E
:10142000E1E7F0E08081816080837894DF91CF9163
:1014300008951F920F920FB60F920BB60F921124C0
:101440002F933F934F935F936F937F938F939F93CC
:10145000AF93BF93EF93FF938091630E9091640ECF
:10146000880F991F880F991F90938700809386009B
:1014700080916D0E813061F0813018F08230A9F4D6
:101480000EC00E94E70890938900809388000DC0E9
:101490000E94E70890938B0080938A0006C00E9408
:1014A000E70890938D0080938C008091730E8130BB
:1014B00061F0813018F08230A9F40EC00E941C093E
:1014C00090938900809388000DC00E941C0990931E
:1014D0008B0080938A0006C00E941C0990938D00A7
:1014E00080938C00FF91EF91BF91AF919F918F916D
:1014F0007F916F915F914F913F912F910F900BBE14
:101500000F900FBE0F901F9018951F920F920FB65D
:101510000F920BB60F9211242F933F934F935F932B
:101520006F937F938F939F93AF93BF93EF93FF93AB
:101530008091650E9091660E880F991F880F991FF4
:10154000909397008093960080916D0E833019F0F0
:10155000843071F407C00E94E7089093990080934B
:10156000980006C00E94E70890939B0080939A0021
:101570008091730E833019F0843071F407C00E949B
:101580001C09909399008093980006C00E941C0942
:1015900090939B0080939A00FF91EF91BF91AF9140
:1015A0009F918F917F916F915F914F913F912F917B
:1015B0000F900BBE0F900FBE0F901F901895519A71
:1015C000509A599A589AE9EBF0E0808183608083C1
:1015D00080E28093B80084E08093BC00089584EAA0
:1015E0008093BC00089584E98093BC00089520E0B6
:1015F00030E002C02F5F3F4F8091BC0087FD06C0E6
:1016000083E228323807B1F780E0089580E028525D
:10161000334208F481E008958093BB0084E880930E
:10162000BC000895813029F48091BC008F70806CDB
:1016300004C08091BC008F7080688093BC000895C6
:101640008091BB0008958091B9000895EF92FF92B8
:101650000F931F93CF93DF93182FE62E042FF52EB1
:1016600084EA8093BC000E94F70A1093BB0084E8D0
:101670008093BC000E94F70A8091B9008871B1F490
:10168000802F9F2D9C01E90110E004E808C089919A
:101690008093BB000093BC000E94F70A1F5F1E15D9
:1016A000B0F384E98093BC0081E004C084E98093B6
:1016B000BC0080E0DF91CF911F910F91FF90EF90E0
:1016C00008950F931F93182F062F84EA8093BC0070
:1016D0000E94F70A1093BB0014E81093BC000E940C
:1016E000F70A8091B900887159F00093BB001093FC
:1016F000BC000E94F70A84E98093BC0081E004C02A
:1017000084E98093BC0080E01F910F910895FF92BF
:101710000F931F93182F062FF42E84EA8093BC009A
:101720000E94F70A1093BB0014E81093BC000E94BB
:10173000F70A8091B900887189F00093BB0010937B
:10174000BC000E94F70AF092BB001093BC000E94FC
:10175000F70A84E98093BC0081E004C084E98093A7
:10176000BC0080E01F910F91FF900895CF92DF920F
:10177000EF92FF921F93CF93DF93182FF62E6A01FB
:1017800084EA8093BC000E94F70A1F5F1093BB009D
:1017900084E88093BC000E94F70A8091B9008871A8
:1017A00059F510E0CF2DD0E021970CC081E00E94C8
:1017B000120B0E94F70A8091BB00F70180830E9400
:1017C000F70A1F5F812F90E07601E80EF91E8C1753
:1017D0009D0764F380E00E94120B0E94F70A80913B
:1017E000BB00F70180830E94F70A84E98093BC0064
:1017F0000E94F70A81E006C084E98093BC000E9441
:10180000F70A80E0DF91CF911F91FF90EF90DF907A
:10181000CF9008950F931F93DF93CF9300D0CDB750
:10182000DEB781E489831A8282E461E08E010F5F72
:101830001F4FA8010E94260B813011F080E006C0E6
:1018400082E462E0A8010E94B60B81E00F900F9045
:10185000CF91DF911F910F9108950F931F93DF9305
:10186000CF9300D0CDB7DEB781E489831A8282E4BA
:1018700061E08E010F5F1F4FA8010E94260B81308F
:1018800029F482E462E0A8010E94B60B998180E00D
:101890002A8130E0282B392BC9010F900F90CF916E
:1018A000DF911F910F9108952F923F924F925F9277
:1018B0006F927F928F929F92AF92BF92CF92DF9260
:1018C000EF92FF920F931F93DF93CF93CDB7DEB7C5
:1018D0002E970FB6F894DEBF0FBECDBFFE01319636
:1018E0008AE0DF011D928A95E9F78EEE64EF4EE201
:1018F0000E94870B813009F588E092E028EC30E007
:10190000F9013197F1F70197D9F78EEE66EF0E9452
:10191000610B813079F48EEE62E0AE014F5F5F4F74
:101920000E94B60B998180E02A81022F10E0082BDB
:10193000192B09C08CE693E002C083E793E00E9474
:101940006A0800E010E08EEE64EF44EF0E94870B1F
:101950008130D1F588E29AE028EC30E0F901319746
:10196000F1F70197D9F78EEE66EF0E94610B813097
:1019700041F58EEE63E0AE014F5F5F4F0E94B60B04
:10198000898190E0A0E0B0E02C01332422248B81F7
:1019900090E0A0E0B0E0282A392A4A2A5B2A9A81FE
:1019A00080E0AA2797FDA095BA2F282A392A4A2A2B
:1019B0005B2A45E055944794379427944A95D1F78C
:1019C0000AC08AE793E002C081E893E00E946A08B7
:1019D000222433242101B801882777FD8095982F90
:1019E0002091B40D3091B50D40E050E0621B730BB7
:1019F000840B950B2091B20D3091B30D40E050E077
:101A00000E9468247B018C013FE015950795F794AF
:101A1000E7943A95D1F76091BC0D7091BD0D882780
:101A200077FD8095982F2BE0660F771F881F991FF1
:101A30002A95D1F72091BE0D3091BF0D442737FD77
:101A40004095542F2E0D3F1D401F511F0E94D02442
:101A500059016A01AE0CBF1CC01ED11E88E090E087
:101A6000A0E0B0E0A80EB91ECA1EDB1ED601C5015B
:101A700014E0B595A795979587951A95D1F790930A
:101A8000A50D8093A40D88E590EFAFEFBFEFA80EF2
:101A9000B91ECA1EDB1EC601B501A60195010E9432
:101AA00068243B014C01ACE095948794779467944B
:101AB000AA95D1F72091AE0D3091AF0D442737FD97
:101AC0004095542FC601B5010E9468247B018C010A
:101AD000FDE015950795F794E794FA95D1F782E024
:101AE00090E0A0E0B0E0E80EF91E0A1F1B1F209155
:101AF000B60D3091B70D442737FD4095542FC401E2
:101B0000B3010E946824BC01992777FD9095892F25
:101B1000E60EF71E081F191F52E015950795F7945A
:101B2000E7945A95D1F780E090E8A0E0B0E0E80EA5
:101B3000F91E0A1F1B1F2091B00D3091B10D40E01E
:101B400050E0C801B7010E946824DC01CB014FE0DE
:101B5000B695A795979587954A95D1F78B879C87DA
:101B6000AD87BE872091AC0D3091AD0D442737FD78
:101B70004095542FC601B5010E9468247B018C0159
:101B80003BE015950795F794E7943A95D1F7809146
:101B9000AA0D9091AB0DAA2797FDA095BA2F22E030
:101BA000880F991FAA1FBB1F2A95D1F7E80EF91EAF
:101BB0000A1F1B1F2091B80D3091B90D442737FD26
:101BC0004095542FC401B3010E946824ABE0959561
:101BD000879577956795AA95D1F7E60EF71E081FAA
:101BE000191FEE0CFF1C001F111F2E183F08400A82
:101BF000510AC201B1012AE638E140E050E00E94FA
:101C0000682497FD0FC0660F771F881F991F2B85CB
:101C10003C854D855E850E94AE24C901DA015C01D8
:101C20006D010CC02B853C854D855E850E94AE24E0
:101C300059016A01AA0CBB1CCC1CDD1C5527D7FC22
:101C40005A954D2D3C2D2B2DCA01B9010E946824B7
:101C50002EED3BE040E050E00E9468247B018C01C7
:101C6000C601B50123E433EE4FEF5FEF0E94682415
:101C7000BC01992777FD9095892F6153714F8F4F44
:101C80009F4F78011127F7FC1095012F6E0D7F1DD6
:101C9000801F911F24E095958795779567952A95E4
:101CA000D1F76A0D7B1D8C1D9D1D6093A60D709351
:101CB000A70D8093A80D9093A90D81E02E960FB6E5
:101CC000F894DEBF0FBECDBFCF91DF911F910F9172
:101CD000FF90EF90DF90CF90BF90AF909F908F904C
:101CE0007F906F905F904F903F902F90089588E87D
:101CF00093E00E946A088091A40D9091A50D6AE07E
:101D000070E00E949B24882777FD8095982F0E9481
:101D100075088FE893E00E946A088091A40D909165
:101D2000A50D6AE070E00E949B24AA2797FDA0956C
:101D3000BA2FBC01CD010E94750881E993E00E9491
:101D40006A088091A40D9091A50D089584E993E00F
:101D50000E946A086091A60D7091A70D8091A80D50
:101D60009091A90D0E94750881E993E00E946A088C
:101D70006091A60D7091A70D8091A80D9091A90D6D
:101D800008950F931F93DF93CF93CDB7DEB72A97B4
:101D90000FB6F894DEBF0FBECDBF8E010F5F1F4F91
:101DA0008AE0F80111928A95E9F78EEE64EF4EE22F
:101DB0000E94870B813011F080E0DAC18EEE6AEA72
:101DC0000E94610B8EEE62E0A8010E94B60B81308A
:101DD00081F4898190E0A0E0B0E0BA2FA92F982F7C
:101DE00088272A8130E0282B392B3093AB0D2093A4
:101DF000AA0D8EEE6CEA0E94610B8EEE62E0AE01DF
:101E00004F5F5F4F0E94B60B813081F4898190E073
:101E1000A0E0B0E0BA2FA92F982F88272A8130E0C0
:101E2000282B392B3093AD0D2093AC0D8EEE6EEA3E
:101E30000E94610B8EEE62E0AE014F5F5F4F0E9429
:101E4000B60B813081F4898190E0A0E0B0E0BA2F38
:101E5000A92F982F88272A8130E0282B392B3093FF
:101E6000AF0D2093AE0D8EEE60EB0E94610B8EEEF7
:101E700062E0AE014F5F5F4F0E94B60B813081F48C
:101E8000898190E0A0E0B0E0BA2FA92F982F882791
:101E90002A8130E0282B392B3093B10D2093B00DDF
:101EA0008EEE62EB0E94610B8EEE62E0AE014F5F40
:101EB0005F4F0E94B60B813081F4898190E0A0E0F1
:101EC000B0E0BA2FA92F982F88272A8130E0282B3D
:101ED000392B3093B30D2093B20D8EEE64EB0E943C
:101EE000610B8EEE62E0AE014F5F5F4F0E94B60B5A
:101EF000813081F4898190E0A0E0B0E0BA2FA92F71
:101F0000982F88272A8130E0282B392B3093B50D64
:101F10002093B40D8EEE66EB0E94610B8EEE62E0B4
:101F2000AE014F5F5F4F0E94B60B813081F4898113
:101F300090E0A0E0B0E0BA2FA92F982F88272A813F
:101F400030E0282B392B3093B70D2093B60D8EEE51
:101F500068EB0E94610B8EEE62E0AE014F5F5F4F57
:101F60000E94B60B813081F4898190E0A0E0B0E05E
:101F7000BA2FA92F982F88272A8130E0282B392BB8
:101F80003093B90D2093B80D8EEE6AEB0E94610B71
:101F90008EEE62E0AE014F5F5F4F0E94B60B813064
:101FA00081F4898190E0A0E0B0E0BA2FA92F982FAA
:101FB00088272A8130E0282B392B3093BB0D2093C2
:101FC000BA0D8EEE6CEB0E94610B8EEE62E0AE01FC
:101FD0004F5F5F4F0E94B60B813081F4898190E0A2
:101FE000A0E0B0E0BA2FA92F982F88272A8130E0EF
:101FF000282B392B3093BD0D2093BC0D8EEE6EEB4C
:102000000E94610B8EEE62E0AE014F5F5F4F0E9457
:10201000B60B813081F4898190E0A0E0B0E0BA2F66
:10202000A92F982F88272A8130E0282B392B30932D
:10203000BF0D2093BE0D8BE993E00E946A0860916A
:10204000AA0D7091AB0D882777FD8095982F0E947F
:10205000750882EA93E00E946A086091AC0D709165
:10206000AD0D882777FD8095982F0E94750882EA2C
:1020700093E00E946A086091AE0D7091AF0D8827C1
:1020800077FD8095982F0E94750882EA93E00E9460
:102090006A086091B00D7091B10D80E090E00E94EF
:1020A000750882EA93E00E946A086091B20D70910F
:1020B000B30D80E090E00E94750882EA93E00E94F0
:1020C0006A086091B40D7091B50D80E090E00E94B7
:1020D000750882EA93E00E946A086091B60D7091DB
:1020E000B70D882777FD8095982F0E94750882EAA2
:1020F00093E00E946A086091B80D7091B90D88272D
:1021000077FD8095982F0E94750882EA93E00E94DF
:102110006A086091BA0D7091BB0D882777FD809594
:10212000982F0E94750882EA93E00E946A086091E5
:10213000BC0D7091BD0D882777FD8095982F0E946A
:10214000750882EA93E00E946A086091BE0D709162
:10215000BF0D882777FD8095982F0E94750882EA29
:1021600093E00E946A0881E993E00E946A0881E096
:102170002A960FB6F894DEBF0FBECDBFCF91DF9188
:102180001F910F910895FC018081860F808308952F
:10219000FC018081819580830895FC018081860FF8
:1021A00080830895FC018081819580830895FC01DE
:1021B00080819181860F971F918380830895FC0110
:1021C00080819181909581959F4F9183808308951F
:1021D000FC0180819181860F971F918380830895F0
:1021E000FC0180819181909581959F4F918380839F
:1021F0000895FC01882777FD8095982F20813181F3
:1022000042815381260F371F481F591F2083318376
:10221000428353830895FC0180819181A281B3811F
:10222000B095A095909581959F4FAF4FBF4F8083FC
:102230009183A283B38308959A9A0895A29A0895E8
:10224000A2980895E42FF0E0DF01A959BF4E1C9237
:10225000DF01AD5ABF4E8C93E15CFF4E108260935C
:10226000DA0D8091D00D8A3F28F48091D00D8F5FD8
:102270008093D00D6623C1F08091D40D9091D50D3F
:1022800066956695262F30E0820F931F9093D50DAB
:102290008093D40D8091D60D9091D70D280F391FC2
:1022A0003093D70D2093D60D8091D40D9091D50DFC
:1022B000855F9140F0F02091D60D3091D70D60915F
:1022C000D40D7091D50D84E690E0AC01249FC0013F
:1022D000259F900D349F900D11240E9487246093B8
:1022E000D30D1092D50D1092D40D1092D70D1092DF
:1022F000D60D08951F920F920FB60F920BB60F9244
:102300001124EF92FF920F931F932F933F934F93BC
:102310005F936F937F938F939F93AF93BF93EF934D
:10232000FF939091C6009093D80D8091060E8093F4
:10233000070E8091050E8093060E8091040E809307
:10234000050E8091030E8093040E9093030E8091EE
:10235000020E882349F4943209F00CC181E0809385
:10236000020E1092010E06C1813009F041C0209189
:10237000010E253031F58091ED0D823551F48091BB
:10238000EE0D8D3401F58091EF0D8334E1F482E0A0
:102390000BC08734C1F48091EE0D873451F48091E5
:1023A000EF0D813481F483E08093020E1092010ED0
:1023B0001AC0833541F48091EF0D813421F484E01B
:1023C000F3CF243170F4E22FF0E0E551F24F908327
:1023D000E22FEF5FE093010EF0E0E551F24F108243
:1023E00002C01092020E1092000E1092FF0DC2C099
:1023F0008230E1F59D3009F4BBC09C3209F0A9C0E0
:10240000F090FF0D83E18F1508F4A3C0E090000E5B
:10241000E4E0EE1639F0F6E0EF1621F082E0E8167F
:1024200009F091C00F2D10E08BEE9DE00E94262553
:10243000000F111F0D551F4EF80191838083F394F7
:10244000F092FF0DEBEEFDE090E080818E3249F4DA
:102450000F2D10E0892F90E08451924F0E94262585
:1024600067C09F5F3196943181F76DC0833009F06A
:1024700047C09D3009F47CC09C3209F06AC0F090DE
:10248000FF0DF3E1FF1508F464C0E090000E85E055
:10249000E81608F458C0E6E0EE1520F4F8E0EF1670
:1024A00009F051C00F2D10E00A5F1F4F8BEE9DE029
:1024B0000E9426259C01000F111F0D551F4EF8018B
:1024C00031832083F394F092FF0D20E030E0822FDF
:1024D000F901E551F24FE081EE23A9F1EE3251F41A
:1024E0000F2D10E00A5F1F4F90E08451924F0E9421
:1024F00026251EC02F5F3F4F2431310541F723C0F1
:102500008430B1F59D30A1F19C3219F5F090FF0DAA
:10251000F3E1FF15F0F0E090000E81E0E81699F489
:102520000F2D10E0065F1F4F8BEE9DE00E942625C9
:102530009C01000F111F0D551F4EF80131832083A0
:10254000F394F092FF0D1092010EE394E092000ECE
:1025500011C0A091010EEA2FF0E0E551F24F9083F7
:10256000AF5FA093010EB0E0A551B24F1C9202C024
:102570001092020EFF91EF91BF91AF919F918F91B9
:102580007F916F915F914F913F912F911F910F918B
:10259000FF90EF900F900BBE0F900FBE0F901F900B
:1025A00018951F920F920FB60F920BB60F9211242F
:1025B0002F933F934F935F936F937F938F939F934B
:1025C000AF93BF93EF93FF93DF93CF9300D000D0EF
:1025D00000D0CDB7DEB75091CE005093D90D909179
:1025E000E90D9093EA0D2091E80D2093E90D3091CB
:1025F000E70D3093E80D4091E60D4093E70D5093C1
:10260000E60D8091E30D823001F58091E50D813377
:1026100009F08DC099832A833B834C835D831E829E
:10262000CE0101960E94222520E030E040E251E4F4
:102630000E9444210E946E1F6115710509F475C046
:102640007093A6106093A51070C08091E30D813047
:1026500009F073C08091E50D823191F499832A834A
:102660003B834C831D821E82CE0101960E9426254B
:10267000009709F45CC09093A4108093A31057C0F6
:10268000873191F499832A833B834C831D821E8278
:10269000CE0101960E942625009709F448C0909328
:1026A000A6108093A51043C08F3189F499832A83A3
:1026B0003B834C835D831E82CE0101960E942625BA
:1026C0000097A9F19093A8108093A71030C084328E
:1026D00089F499832A833B834C835D831E82CE01D8
:1026E00001960E942625009711F19093AA108093DD
:1026F000A9101DC08B32D9F499832A833B834C8364
:102700005D831E82CE0101960E94222520E030E0EA
:1027100048EC52E40E9444210E946E1F611571052D
:1027200021F07093AC106093AB101092E30D809188
:10273000E50D8F5F8093E50D2CC09734B9F42035FB
:10274000A9F4323541F44D3489F4533479F41092BC
:10275000E50D81E009C0373449F4473439F4513488
:1027600029F41092E50D82E08093E30D8091E90D4C
:10277000823B79F48091E80D853A59F48091E70D18
:10278000853639F45B3429F4F89480E00E94EB0339
:10279000FFCF2696DEBFCDBFCF91DF91FF91EF91A6
:1027A000BF91AF919F918F917F916F915F914F9169
:1027B0003F912F910F900BBE0F900FBE0F901F9067
:1027C0001895CF92DF92EF920F93CF93DF936C0126
:1027D000EE2DF0E0DF01A959BF4E6C93DF01AD5A39
:1027E000BF4E4C93E15CFF4E20830093DA0DFC0159
:1027F00080819181A281B3818093DC0D9093DD0D66
:10280000A093DE0DB093DF0D1092D00D8091D40D0A
:102810009091D50D01969093D50D8093D40D002302
:10282000C1F08091D40D9091D50D202F269526953D
:1028300030E0820F931F9093D50D8093D40D80913B
:10284000D60D9091D70D280F391F3093D70D2093B7
:10285000D60D8091D40D9091D50D855F9140F0F00B
:102860002091D60D3091D70D6091D40D7091D50D7A
:1028700084E690E0AC01249FC001259F900D349F19
:10288000900D11240E9487246093D30D1092D50DD2
:102890001092D40D1092D70D1092D60DD601149629
:1028A0008C911497813009F086C088E08093D20D16
:1028B00058968D919C91599790930A0E8093090E8A
:1028C000E0E010C0F0E0DF011496AA0FBB1FAC0DD2
:1028D000BD1D8D919C91EE0FFF1FE558FF4E91831A
:1028E0008083E22F8091D20D2E2F2F5FE81750F3B7
:1028F000E093080EF60186818F3F39F487818823A3
:1029000021F080931F0D1092D10D1092080E24C05B
:10291000C22FD0E0FE01EE0FFF1FDF01A558BF4E12
:102920008D919C91E957F14F91838083253078F404
:10293000C55DD14FE88DF0E0EE0FFF1FE558FF4E6B
:1029400060817181660F771F822F0E945A098091E2
:10295000080E8F5F8093080E2091080E8091D20D93
:102960002817B0F2D60116968C9116978093C60D53
:1029700016968C911697E82FF0E08091D20D9F016A
:10298000280F311D2034310594F48091D20DE80FC9
:10299000F11D17968C9124E1829FC00111248C5E59
:1029A0009940EE0FFF1FE957F14F9183808381E03B
:1029B0008093E40D86C0823009F083C080E180936B
:1029C000D20DD60198968D919C91999790930A0E6D
:1029D0008093090EE0E010C0F0E0DF011496AA0F2A
:1029E000BB1FAC0DBD1D8D919C91EE0FFF1FE558D7
:1029F000FF4E91838083E22F8091D20D2E2F2F5F87
:102A0000E81750F3E093080EF60186818F3F39F402
:102A10008781882321F080931F0D1092D10D109291
:102A2000080E24C0C22FD0E0FE01EE0FFF1FDF0111
:102A3000A558BF4E8D919C91E957F14F91838083AA
:102A4000253078F4C55DD14FE88DF0E0EE0FFF1F23
:102A5000E558FF4E60817181660F771F822F0E94BB
:102A60005A098091080E8F5F8093080E2091080EFE
:102A70008091D20D2817B0F2D60116968C91169738
:102A80008093C60D16968C911697E82FF0E08091F2
:102A9000D20D9F01280F311D2034310594F480910F
:102AA000D20DE80FF11D17968C9124E1829FC00191
:102AB00011248C5E9940EE0FFF1FE957F14F91836F
:102AC00080838091090E8093DB0D8091C40D8B3043
:102AD00030F584E0D60114968C9314978091C40D40
:102AE00015968C93159716961C928091C40D90E0C4
:102AF0002AE130E0829FF001839FF00D929FF00D5C
:102B00001124E95FF04F178A6091C40D8AE1689F34
:102B1000B0011124695F704FC601089614C08091FE
:102B2000C40D8C3028F584E0D60114968C9314974C
:102B30008091C40D15968C93159716961C92C6011C
:102B4000089669EA73E00E944F258091090E9091E2
:102B50000A0EF60191A380A3019690930A0E80932A
:102B6000090E8091C40D8F5F8093C40D84E2D4C0A0
:102B70008091C40D8F5F8093C40D8150853110F01A
:102B80001092C40D83E0D60114968C931497809113
:102B9000200D15968C9315978091090E90910A0E31
:102BA00019969C938E931897019690930A0E809392
:102BB000090E8091200D813188F4893008F070C0B1
:102BC0008330A9F1843030F48130F1F0823009F0A3
:102BD00098C01EC0843009F05EC042C0833109F441
:102BE00077C0843138F4813109F465C0823109F04D
:102BF00088C069C0853109F475C0853108F46DC09D
:102C0000863109F07EC073C0F601068317827EC04C
:102C100020E030E090E008C0E92FF0E0E959FF4EF5
:102C20008081280F311D9F5F9031B0F327C020E0D5
:102C300030E090E008C0E92FF0E0ED5AFF4E8081CF
:102C4000280F311D9F5F9031B0F39093080E74E010
:102C5000369527957A95E1F7F6013783268356C096
:102C600020E030E090E008C0E92FF0E0E15CFF4EAA
:102C70008081280F311D9F5F9031B0F39093080E33
:102C800064E0369527956A95E1F7D60117963C934F
:102C90002E9316973BC090E005970E94D2080FC074
:102CA000E82FF0E0EE0FFF1FEF5DF14F8081918183
:102CB0008051984F20C08091A3109091A410F601EC
:102CC0009783868323C08091A5109091A61013C08E
:102CD0008091A7109091A810F2CF8091A9109091A7
:102CE000AA1009C08091AB109091AC10E8CF8091F0
:102CF000AD109091AE10D60117969C938E931697B7
:102D000005C0F601868317821092200D8091200D58
:102D10008F5F8093200D8CE0DF91CF910F91EF902A
:102D2000DF90CF90089588EB93E00E946A080895A1
:102D3000CF93DF938BEE93E00E946A08C0E0D0E06F
:102D40008FEE93E00E946A08FE01ED5AFF4E8081EB
:102D500090E00E94A0082196C031D10589F781EF4B
:102D600093E00E946A08C0E0D0E08FEE93E00E94FA
:102D70006A08FE01E959FF4E808190E00E94A00898
:102D80002196C031D10589F788EF93E00E946A0847
:102D9000C0E0D0E08FEE93E00E946A08FE01E15CA3
:102DA000FF4E808190E00E94A0082196C031D1059D
:102DB00089F78FEF93E00E946A088FEE93E00E94FC
:102DC0006A0880E090E00E94D2080E94A0088FEE7E
:102DD00093E00E946A0881E090E00E94D2080E947D
:102DE000A0088FEE93E00E946A0882E090E00E94C3
:102DF000D2080E94A0088FEE93E00E946A0883E048
:102E000090E00E94D2080E94A00886E094E00E9410
:102E10006A08C0E0D0E08FEE93E00E946A08FE01ED
:102E2000EE0FFF1FE558FF4E808191810E94A008A0
:102E30002196C031D10579F78DE094E00E946A08AF
:102E4000C0E0D0E08FEE93E00E946A08FE01EE0F32
:102E5000FF1FED5CF14F808191810E94A0082196B7
:102E6000C830D10579F784E194E00E946A08809126
:102E7000DA0D90E00E94A0088FEE93E00E946A08AD
:102E80008091D60D9091D70D0E94A0088FEE93E00F
:102E90000E946A088091D40D9091D50D0E94A008DF
:102EA0008FEE93E00E946A088091D30D90E00E941B
:102EB000A0088FEE93E00E946A088091DC0D90914B
:102EC000DD0DA091DE0DB091DF0D0E94A0088FEE08
:102ED00093E00E946A0880912B0E90912C0EA09195
:102EE0002D0EB0912E0E0E94A0088FEE93E00E944E
:102EF0006A088091DB0D90E00E94A0088CE194E0CC
:102F00000E946A08C0E0D0E08FEE93E00E946A0859
:102F1000FE01EE0FFF1FED55FF4E808191810E9453
:102F2000A0082196CB30D10579F783E294E00E9486
:102F30006A08DF91CF9108950F931F93CF93DF938A
:102F40008FEF0E9460068FEF0E94600640E050E025
:102F500020E030E0F901E959FF4E8081480F511D12
:102F60002F5F3F4F20313105A9F7A4E056954795D3
:102F7000AA95E1F7842F0E94600640E050E020E02F
:102F800030E0F901E15CFF4E8081480F511D2F5F59
:102F90003F4F20313105A9F7F5E056954795FA9551
:102FA000E1F7842F0E946006C0E0D0E08E01000FA0
:102FB000111F05581F4EF801808191818050984F54
:102FC000892F0E946006F801808191810E9460062D
:102FD0002196C031D10551F7DF91CF911F910F910B
:102FE0000895CF93DF938FEF0E9460068FEF0E94CA
:102FF000600640E050E020E030E0F901E959FF4E82
:103000008081480F511D2F5F3F4F20313105A9F7B7
:1030100094E0569547959A95E1F7842F0E946006B3
:1030200040E050E020E030E0F901E15CFF4E8081BB
:10303000480F511D2F5F3F4F20313105A9F785E023
:10304000569547958A95E1F7842F0E946006C0E067
:10305000D0E0FE01EE0FFF1FE558FF4E8081918109
:103060008050984F60E170E00E949B24862F0E9460
:1030700060062196C031D10561F7DF91CF910895A7
:103080000F931F93DF93CF9300D00F92CDB7DEB78E
:103090008BE189838BE58A838AE48B838E010F5FC2
:1030A0001F4FC80163E00E94090682E089831A82EB
:1030B000C80162E00E9409060F900F900F90CF9117
:1030C000DF911F910F9108950F931F93DF93CF937B
:1030D00000D000D0CDB7DEB78BE189838BE58A8342
:1030E0008BE38B8388E48C838E010F5F1F4FC801B5
:1030F00064E00E94090682E089831A82C80162E0C6
:103100000E9409060F900F900F900F90CF91DF91C2
:103110001F910F9108951F93CF93DF930E94401842
:103120000E94641887E294E00E946A0882E694E0B4
:103130000E946A088FE894E00E946A0886EC94E096
:103140000E946A0885ED94E00E946A0880916D0EE5
:10315000803150F58EED94E00E946A0880916E0EE9
:1031600090E00E94A00886EE94E00E946A08809198
:103170006D0E90E001960E94A00887EF94E00E94F7
:103180006A0880916F0E90E00E94A0088AEF94E098
:103190000E946A088091700E9091710E0E94A008A2
:1031A0008CEF94E00E946A0881E095E00E946A0832
:1031B0008DE095E00E946A0887E195E00E946A0828
:1031C00089E295E00E946A0888E395E00E946A0817
:1031D0008EE395E00E946A0884E495E00E946A0804
:1031E0008AE495E00E946A0887E195E00E946A08F7
:1031F0008EE595E00E946A08C0E0D0E013E0FE0191
:10320000E959FF4E8081819FC00111248B55904068
:103210000E94A0088DE695E00E946A082196C031C0
:10322000D10569F78FE695E00E946A08C0E0D0E01A
:1032300013E0FE01ED5AFF4E8081819FC0011124F1
:103240008B5590400E94A0088DE695E00E946A0888
:103250002196C031D10569F78FE895E00E946A0890
:10326000C0E0D0E013E0FE01ED5AFF4E4081FE01C8
:10327000E959FF4E8081819FC001112450E09A01DD
:10328000220F331F240F351F821B930B0E94A008AF
:103290008DE695E00E946A082196C031D10519F7A4
:1032A0008FEA95E00E946A08C0E0D0E0FE01E15C90
:1032B000FF4E808190E00E94A0088DE695E00E947C
:1032C0006A082196C031D10589F78FEC95E00E94FC
:1032D0006A088091DA0D90E00E94A0088FEE95E0D8
:1032E0000E946A088091D60D9091D70D0E94A00887
:1032F00081EF95E00E946A088091D40D9091D50DE0
:103300000E94A00883EF95E00E946A088091D30D87
:1033100090E00E94A00885EF95E00E946A088091E5
:103320002C0D90912D0D0E94A00881EF95E00E9438
:103330006A0880912202909123020E94A00887E1EE
:1033400096E00E946A088091DC0D9091DD0DA091BD
:10335000DE0DB091DF0D0E94A00889E396E00E9487
:103360006A0880912B0E90912C0EA0912D0EB09199
:103370002E0E0E94A0088CE396E00E946A088091BD
:10338000DB0D90E00E94A0088DE596E00E946A089F
:103390008CE696E00E946A0880E090E00E94D208E5
:1033A0000E94A0088DE796E00E946A0881E090E004
:1033B0000E94D2080E94A00881E896E00E946A0854
:1033C00082E090E00E94D2080E94A00885E896E082
:1033D0000E946A0883E090E00E94D2080E94A00840
:1033E00089E896E00E946A0880E996E00E946A08EF
:1033F0008091660090E00E94A0088FE996E00E940C
:103400006A0889EA96E00E946A0880912F0E90E08F
:103410000E94A00888EB96E00E946A088091300E16
:1034200090E00E94A0088FE996E00E946A088BEB6A
:1034300096E00E946A0810E00FC0E12FF0E0EE0F66
:10344000FF1FE558FF4E808191810E94A0088DE604
:1034500095E00E946A081F5F8091D20D181768F3EB
:103460008FE996E00E946A088AEC96E00E946A085A
:103470008091C60D992787FD90950E94A0088FE93D
:1034800096E00E946A0889ED96E00E946A088FEE35
:1034900095E00E946A088091720E90E00E94A00858
:1034A00088EE96E00E946A088091720E20916E0E5E
:1034B00090E0820F911D0E94A0088BEE96E00E9482
:1034C0006A0810E011C08091720EE80FF11DEE0F36
:1034D000FF1FE957F14F808191810E94A0088DE67E
:1034E00095E00E946A081F5F80916E0E181750F4D5
:1034F000E12FF0E08091720E9F01280F311D2034E2
:1035000031050CF38EEE96E00E946A088FEE95E08E
:103510000E946A088091780E90E00E94A00888EED0
:1035200096E00E946A088091780E2091740E90E0D7
:10353000820F911D0E94A0088BEE96E00E946A08FF
:1035400010E011C08091780EE80FF11DEE0FFF1F03
:10355000E957F14F808191810E94A0088DE695E0A6
:103560000E946A081F5F8091740E181750F4E12FB3
:10357000F0E08091780E9F01280F311D2034310535
:103580000CF38FE996E00E946A08DF91CF911F91BA
:1035900008950F93FC0101900020E9F73197E81B93
:1035A000F90BDB016D917C918E0F9F1F40E020E0B5
:1035B00001E00E94F7060F9108950F93FC0101901E
:1035C0000020E9F73197E81BF90BDB016D917C9145
:1035D0008E0F9F1F40E020E001E00E94F7060F9150
:1035E00008950F93FC0101900020E9F73197E81B43
:1035F000F90BDB016D917C918E0F9F1F40E020E065
:1036000001E00E94F7060F9108950F93DC010D90E1
:103610000020E9F71197A81BB90BFB016081772700
:1036200067FD70958A0F9B1F40E020E001E00E943B
:10363000F7060F9108950F93FC0101900020E9F720
:103640003197E81BF90BDB016C918E0F9F1F70E027
:1036500040E020E001E00E94F7060F9108958F926C
:103660009F92AF92BF92CF92DF92EF92FF920F9311
:103670001F93DF93CF93CDB7DEB7A0970FB6F89423
:10368000DEBF0FBECDBF282F19824091C10D909192
:10369000C00DA92FB0E0FD01E751F34FE081BE2E30
:1036A000B40E8091790E882319F481E08093790E0D
:1036B000233309F46AC0243338F4213309F4ACC04D
:1036C000223309F0BCC013C0263329F1283321F07E
:1036D000243309F0B4C060C0442311F0415012C03B
:1036E000AC50B34F8C9181508093C10D10C0242FEA
:1036F00030E0AC50B34F8C9190E001972817390718
:1037000024F44F5F4093C10D02C01092C10DB090E0
:10371000C10DBE0E94C0AB2DB0E0FD01EF53F84FCC
:10372000E081E230F9F0E33030F4EE23D9F0E1301B
:1037300009F085C008C0E430F9F0E430E8F0E53085
:1037400009F07DC022C0AA0FBB1FAE5FB74FED913D
:10375000FC9180819181A281B3818C509E4FAF4FAB
:10376000BF4F4BC0AA0FBB1FAE5FB74FED91FC918F
:10377000808191810A9630C0AA0FBB1FAE5FB74F00
:10378000ED91FC9180818F5F45C09A3010F49F5F6E
:1037900046C01092C00D49C0AB2DB0E0FD01EF5303
:1037A000F84FE081E23079F0E33030F4EE2359F065
:1037B000E13009F044C013C0E43021F1E43010F1ED
:1037C000E530E9F529C0AA0FBB1FAE5FB74FED91F9
:1037D000FC91808191810A979183808330C0AA0FE8
:1037E000BB1FAE5FB74FED91FC9180819181A281AB
:1037F000B381845F9140A040B04080839183A283D5
:10380000B3831DC0AA0FBB1FAE5FB74FED91FC91F4
:1038100080818150808313C0992321F0915090932F
:10382000C00D03C08AE08093C00D1092C10DE091DD
:10383000C00DF0E0E751F34FB080B092C20D0B2DF8
:1038400010E02091C20D8091790E90E0820F911DC1
:103850000197081719074CF08091790E2B2D281B22
:10386000822F8F5F8093C20D04C0B21610F4B09205
:10387000C20D86E097E00E946A08E091C00DF0E07A
:10388000E751F34F208181E090E0821B9109800F86
:10389000911F0E94A00881EF95E00E946A08E091C4
:1038A000C00DF0E0EC50F34F808190E00E94A00842
:1038B0008AE097E00E946A08E091C00DF0E0EE0F08
:1038C000FF1FED52F34F808191810E946A088CE0C6
:1038D00097E00E946A0881E197E00E946A08E091FF
:1038E000C00DF0E0EE0FFF1FED52F34F60817181CC
:1038F0008BE090E10E944F2500E010E0C801895F55
:10390000904F63EF75E00E944F25065E1F4F31E038
:103910000430130799F7A090C20D7E010894E11CB2
:10392000F11CEAE18E2E912C89C01982BA1429F477
:10393000C70169E277E00E9444258601000F111F4C
:10394000F801E251F44F60817181C7010E94442562
:10395000C7016BE277E00E944425F601EF53F84F70
:10396000E081E23001F1E33028F4EE2351F0E13060
:10397000C1F510C0E43039F1E430F0F0E53089F5FC
:103980002BC00E5F174FF80160817181C7010E9443
:10399000DD1A27C00E5F174FF80160817181C701E2
:1039A0000E94C91A1EC00E5F174FF8016081718115
:1039B000C7010E94F11A15C00E5F174FF801608110
:1039C0007181C7010CC00E5F174FF80160817181D2
:1039D000C7010E94051B05C0C70160EC7DE00E9485
:1039E0001B1B8DE297E00E946A088091C20D960130
:1039F000281B3109C9010E94A0088AE097E00E94B3
:103A00006A08C7010E946A0881E397E00E946A0879
:103A10008091C20DF601E81BF109EA30F1056CF462
:103A2000188EE89DC001E99D900DF89D900D112420
:103A3000895F904FB7010E944F25A394CA2CDD24C3
:103A40002091790E8091C20D90E0820F911DC816D1
:103A5000D906A4F430E43A1588F0E091C00DF0E006
:103A6000DF01AC50B34F2C91E751F34F808190E0D0
:103A7000820F911DC816D9060CF457CF81E197E04B
:103A80000E946A08A0960FB6F894DEBF0FBECDBFA5
:103A9000CF91DF911F910F91FF90EF90DF90CF902A
:103AA000BF90AF909F908F900895AF92BF92CF92AA
:103AB000DF92EF92FF920F931F93CF93DF931092B9
:103AC000C30D1092C50D80E090E02AE130E0829FA6
:103AD000F001839FF00D929FF00D1124E95FF04FEC
:103AE000108201968A30910591F79A9AA29A80E005
:103AF00090E0FC01EE0FFF1FE558FF4E118210828F
:103B0000019680319105A9F780E090E020E80FB69A
:103B1000F89420936100809361000FBE809166004D
:103B2000875F80936600399A419A579A5F9A6B9A99
:103B3000739804B603FC03C081E08093E20D1092F9
:103B4000E20D6E98769A60E076E980E090E00E945F
:103B5000C10584E397E00E946A0888EB93E00E9425
:103B60006A0860E875E280E090E00E94E5050E9446
:103B7000DF0A0E94C7080E949A030E94B40980E0ED
:103B80000E942F1BAA24AA9401E0B3E0FB2EA4E01C
:103B9000EA2EF4ECCF2EF9E0DF2EE2E0BE2E90917B
:103BA0001F0DA0921F0D9F3F09F45AC08091D10DA7
:103BB000882309F055C0992309F452C0892F0E9427
:103BC0002F1B8091320E882309F11092320E81E66C
:103BD00097E00E946A0820E030E0F901EE0FFF1F35
:103BE000E558FF4E80819181F901EE0FFF1FED5CDA
:103BF000F14F918380832F5F3F4F2830310569F764
:103C00000E9405038BE797E00E946A0880917C0E72
:103C10008823C1F010927C0E89E897E00E946A0820
:103C2000F0926D0E1092720EE092730E1092780E5A
:103C3000D092660EC092650E0E9405038BE797E056
:103C40000E946A0880917B0E882341F010927B0EBF
:103C50000E9405038BE797E00E946A080093D10D4C
:103C6000A8958091D90D882371F48091E00D813061
:103C700051F08091E40D813009F0D7C08091E10DC1
:103C8000853009F0D2C01091D90D1092D90D13369C
:103C900019F4B092E10D04C0123429F4F092E10D50
:103CA0000093E00D52C01D3619F41092E10DF8CFCB
:103CB0001636C1F420E030E0F901EE0FFF1FE558A1
:103CC000FF4E80819181F901EE0FFF1FED5CF14FF6
:103CD000918380832F5F3F4F2830310569F70E9421
:103CE000050333C0133721F0812F80538A3028F425
:103CF0000093E10D1092E00D28C0133529F40E94C5
:103D000005038EE997E01FC0123619F40E94AA003D
:103D10001CC0153739F48091E00D902F981B9093BB
:103D2000E00D13C0123759F40E9464188AEA97E034
:103D30000E946A08F89480E00E94EB03FFCF1934D8
:103D400021F488EB93E00E946A088091E10D8230B3
:103D500009F463C0833030F4882359F0813009F0CE
:103D600064C00AC0833009F45BC0843009F05DC0D0
:103D70005AC00E948B1859C0812F0E942F1B80911E
:103D8000320E882309F11092320E81E697E00E94EC
:103D90006A0820E030E0F901EE0FFF1FE558FF4E02
:103DA00080819181F901EE0FFF1FED5CF14F91834E
:103DB00080832F5F3F4F2830310569F70E9405034C
:103DC0008BE797E00E946A0880917C0E8823C1F0FF
:103DD00010927C0E89E897E00E946A08F0926D0EBE
:103DE0001092720EE092730E1092780ED092660EC0
:103DF000C092650E0E9405038BE797E00E946A0857
:103E000080917B0E882389F010927B0E0E9405031F
:103E10008BE797E00E946A0808C00E94981605C0C8
:103E20000E94F11702C00E949C17669906C086EB9B
:103E300097E00E946A080E94AA008091D00D882312
:103E400011F41092CF0D9091310E913009F0A7CE60
:103E50008091D00D853608F4A2CE9093CF0DC0E0AE
:103E6000D0E0FE01EE0FFF1FED5CF14F80819181EC
:103E7000FE01EE0FFF1FE558FF4E91838083C53092
:103E800040F5DE01A55DB14F5896EC915897F0E0F2
:103E9000EE0FFF1FE558FF4E6081718190962C91C7
:103EA000882777FD8095982F332727FD3095432F5E
:103EB000532F0E94682424E630E040E050E00E9446
:103EC000AE24220F331F441F551F8C2FB9010E94AF
:103ED0005A092196C830D10521F661CEEF92FF92A2
:103EE0000F931F937B018C0120E030E040E05FE402
:103EF0000E943E2288238CF0C801B70120E030E008
:103F000040E05FE40E94E6200E946E229B01AC012B
:103F1000205030404040504806C0C801B7010E94C0
:103F20006E229B01AC01B901CA011F910F91FF9054
:103F3000EF900895A0E0B0E0E0EAFFE10C94EB24FC
:103F4000DC012B01FA019C91923008F439C1EB019C
:103F50008881823008F433C1943069F4843009F0E8
:103F60002FC111969C9111978981981709F428C146
:103F7000A1E2BDE025C1843009F421C18230A9F459
:103F8000923009F01DC19A01AD0188E0EA01099063
:103F9000AE01E90109929E018150C1F7E2018981D8
:103FA00011969C918923818308C1923009F407C13D
:103FB00012962D903C901397EB018A819B81149669
:103FC000AD90BD90CD90DC901797EC80FD800E8178
:103FD0001F819101281B390BB90137FF04C06627E7
:103FE0007727621B730B603271050CF061C01216EB
:103FF00013066CF537014801062E04C09694879489
:10400000779467940A94D2F721E030E040E050E0E2
:1040100004C0220F331F441F551F6A95D2F7215049
:104020003040404050402E213F2140235123211554
:1040300031054105510521F021E030E040E050E03C
:1040400079018A01E628F728082919293CC0232B81
:10405000D1F1260E371E35014601062E04C0969476
:104060008794779467940A94D2F721E030E040E097
:1040700050E004C0220F331F441F551F6A95D2F72A
:1040800021503040404050402A213B214C215D21AD
:10409000211531054105510521F021E030E040E0D6
:1040A00050E059016A01A628B728C828D9280BC0B2
:1040B000821593052CF01C01AA24BB24650103C0C2
:1040C000EE24FF24870111969C91D20111968C91C8
:1040D000981709F445C0992339F0A80197012A19C6
:1040E0003B094C095D0906C0A60195012E193F093F
:1040F000400B510B57FD08C011823382228224836A
:104100003583468357831DC081E0818333822282B9
:1041100088279927DC01821B930BA40BB50B8483A2
:104120009583A683B7830DC0220F331F441F551FED
:1041300024833583468357838281938101979383B8
:1041400082832481358146815781DA01C901019733
:10415000A109B1098F5F9F4FAF4FBF4328F30BC039
:10416000918333822282EA0CFB1C0C1D1D1DE4820C
:10417000F5820683178383E080832481358146811D
:10418000578157FF1AC0C901AA2797FDA095BA2FDA
:1041900081709070A070B0705695479537952795AF
:1041A000822B932BA42BB52B84839583A683B78373
:1041B00082819381019693838283DF0101C0D201C2
:1041C000CD01CDB7DEB7E2E10C940725A0E2B0E067
:1041D000ECEEF0E20C94F72469837A838B839C8362
:1041E0002D833E834F835887E9E0EE2EF12CEC0EB1
:1041F000FD1ECE010196B7010E9497238E010F5E2E
:104200001F4FCE010596B8010E9497238A8991E03D
:1042100089278A8BC701B801AE01475E5F4F0E94B4
:104220009A1F0E94C222A096E6E00C941325A0E2F9
:10423000B0E0EDE1F1E20C94F72469837A838B839B
:104240009C832D833E834F835887F9E0EF2EF12C1A
:10425000EC0EFD1ECE010196B7010E9497238E0140
:104260000F5E1F4FCE010596B8010E949723C7012C
:10427000B801AE01475E5F4F0E949A1F0E94C222A2
:10428000A096E6E00C941325A0E2B0E0EAE4F1E2A7
:104290000C94EB2469837A838B839C832D833E83E8
:1042A0004F835887CE010196BE01675F7F4F0E9402
:1042B0009723CE010596BE016F5E7F4F0E94972324
:1042C0009985923088F089898230C8F0943019F449
:1042D000823051F404C0843029F4923081F481E2B8
:1042E0009DE0C6C0923049F420E09A858A899813EF
:1042F00021E02A87CE010996BBC0823049F420E034
:104300009A858A89981321E02A8BCE014196B0C004
:104310002D843E844F8458886D887E888F88988C41
:10432000EE24FF248701AA24BB24650140E050E06D
:1043300060E070E0E0E0F0E0C10181709070892BF6
:10434000E9F0E60CF71C081D191D9A01AB012A0DB6
:104350003B1D4C1D5D1D80E090E0A0E0B0E0E61448
:10436000F7040805190520F481E090E0A0E0B0E032
:10437000BA01A901480F591F6A1F7B1FAA0CBB1C59
:10438000CC1CDD1C97FE08C081E090E0A0E0B0E00E
:10439000A82AB92ACA2ADB2A3196E032F10549F067
:1043A000660C771C881C991C569447943794279464
:1043B000C3CFFA85EA892B893C898B859C85280F98
:1043C000391F2E5F3F4F17C0CA0181709070892B33
:1043D00061F016950795F794E79480E090E0A0E0EF
:1043E000B0E8E82AF92A0A2B1B2B76956795579592
:1043F00047952F5F3F4F77FDE7CF0CC0440F551F08
:10440000661F771F17FD4160EE0CFF1C001F111F78
:1044100021503040403090E0590790E0690790E427
:10442000790760F32B8F3C8FDB01CA018F77907087
:10443000A070B07080349105A105B10561F447FD0D
:104440000AC0E114F1040105110529F0405C5F4F39
:104450006F4F7F4F40781A8EFE1711F081E08A8FE0
:104460004D8F5E8F6F8F78A383E0898FCE01499641
:104470000E94C222A096E2E10C940725A8E1B0E0D8
:10448000E4E4F2E20C94F72469837A838B839C83BF
:104490002D833E834F83588789E0E82EF12CEC0E64
:1044A000FD1ECE010196B7010E9497238E010F5E7B
:1044B0001F4FCE010596B8010E949723898582304F
:1044C00040F08989823028F0C701B8010E940F248A
:1044D00001C08FEF6896E6E00C941325ACE0B0E0E5
:1044E000E4E7F2E20C94FB2469837A838B839C8358
:1044F000CE010196BE016B5F7F4F0E9497238D8195
:10450000823061F1823050F1843021F48E81882331
:1045100051F12EC02F81388537FD20C06E812F319B
:1045200031051CF06623F9F023C08EE190E0821B78
:10453000930B29853A854B855C8504C05695479534
:10454000379527958A95D2F76623B1F05095409517
:10455000309521953F4F4F4F5F4F0EC020E030E028
:1045600040E050E009C02FEF3FEF4FEF5FE704C09E
:1045700020E030E040E050E8B901CA012C96E2E0CA
:104580000C941725DF92EF92FF920F931F93FC017B
:10459000E480F58006811781D1808081823048F4E3
:1045A00080E090E0A0E1B0E0E82AF92A0A2B1B2B7A
:1045B000A5C0843009F49FC0823021F4EE24FF248A
:1045C000870105C0E114F1040105110519F4E0E0CB
:1045D000F0E096C0628173819FEF623879070CF03A
:1045E0005BC022E83FEF261B370B2A3131052CF048
:1045F00020E030E040E050E02AC0B801A701022EE0
:1046000004C076956795579547950A94D2F781E04F
:1046100090E0A0E0B0E004C0880F991FAA1FBB1F64
:104620002A95D2F70197A109B1098E219F21A023D4
:10463000B1230097A105B10521F081E090E0A0E051
:10464000B0E09A01AB01282B392B4A2B5B2BDA0106
:10465000C9018F779070A070B07080349105A1056A
:10466000B10539F427FF09C0205C3F4F4F4F5F4F22
:1046700004C0215C3F4F4F4F5F4FE0E0F0E020303F
:10468000A0E03A07A0E04A07A0E45A0710F0E1E0F2
:10469000F0E079018A0127C06038710564F5FB01FB
:1046A000E158FF4FD801C7018F779070A070B070AC
:1046B00080349105A105B10539F4E7FE0DC080E411
:1046C00090E0A0E0B0E004C08FE390E0A0E0B0E0B4
:1046D000E80EF91E0A1F1B1F17FF05C01695079548
:1046E000F794E794319687E016950795F794E79449
:1046F0008A95D1F705C0EE24FF248701EFEFF0E0A3
:104700006E2F679566276795902F9F77D794DD2446
:10471000D7948E2F8695492F462B582F5D29B701A8
:10472000CA011F910F91FF90EF90DF900895FC0157
:10473000DB01408151812281622F6F7770E0221F5F
:104740002227221F9381892F880F822B282F30E068
:10475000991F9927991F11969C931197211531053F
:10476000A9F5411551056105710511F482E037C0C5
:1047700082E89FEF13969C938E9312979A01AB0158
:1047800067E0220F331F441F551F6A95D1F783E05E
:104790008C930DC0220F331F441F551F12968D910D
:1047A0009C911397019713969C938E9312972030A8
:1047B00080E0380780E0480780E4580758F31496F3
:1047C0002D933D934D935C93179708952F3F31059B
:1047D00079F4411551056105710519F484E08C9354
:1047E000089564FF03C081E08C9312C01C9210C036
:1047F0002F57304013963C932E93129783E08C935F
:1048000087E0440F551F661F771F8A95D1F77064A4
:1048100014964D935D936D937C93179708951F9312
:10482000DC01FB019C91923008F447C0808182300A
:1048300008F443C0943051F411961C91843099F5DA
:104840008181682F70E0611B71093FC0843021F0C5
:10485000923031F48230B9F18181882389F12DC001
:1048600011961C9111978230F1F081811817D9F4BB
:1048700012962D913C911397828193818217930711
:1048800094F028173907BCF014968D919D910D90E6
:10489000BC91A02D24813581468157812817390785
:1048A0004A075B0718F4112341F00AC082179307E7
:1048B000A407B50740F4112319F061E070E005C0CA
:1048C0006FEF7FEF02C060E070E0CB011F910895B1
:1048D000629FD001739FF001829FE00DF11D649FE4
:1048E000E00DF11D929FF00D839FF00D749FF00D70
:1048F000659FF00D9927729FB00DE11DF91F639F11
:10490000B00DE11DF91FBD01CF0111240895AA1BAF
:10491000BB1B51E107C0AA1FBB1FA617B70710F0AA
:10492000A61BB70B881F991F5A95A9F780959095DC
:10493000BC01CD01089597FB092E07260AD077FD0B
:1049400004D0E5DF06D000201AF4709561957F4F02
:104950000895F6F7909581959F4F0895A1E21A2E3C
:10496000AA1BBB1BFD010DC0AA1FBB1FEE1FFF1F13
:10497000A217B307E407F50720F0A21BB30BE40B63
:10498000F50B661F771F881F991F1A9469F76095AA
:104990007095809590959B01AC01BD01CF01089564
:1049A00097FB092E05260ED057FD04D0D7DF0AD07D
:1049B000001C38F450954095309521953F4F4F4F4E
:1049C0005F4F0895F6F790958095709561957F4FAC
:1049D0008F4F9F4F08952F923F924F925F926F9209
:1049E0007F928F929F92AF92BF92CF92DF92EF927F
:1049F000FF920F931F93CF93DF93CDB7DEB7CA1B00
:104A0000DB0B0FB6F894DEBF0FBECDBF09942A882A
:104A1000398848885F846E847D848C849B84AA84D2
:104A2000B984C884DF80EE80FD800C811B81AA815F
:104A3000B981CE0FD11D0FB6F894DEBF0FBECDBF2A
:104A4000ED010895662777270C948625FC018827B9
:104A50009927E89421912032E9F3293010F02E3083
:104A6000C8F32B3241F02D3239F4689404C00E940F
:104A70005625820F911D219120532A30C0F31EF438
:104A8000909581959F4F0895FB01DC010D900020CA
:104A9000E9F7119701900D920020E1F70895FB01CD
:104AA000DC0101900D920020E1F708957AE0979FD4
:104AB000902D879F802D910D11240895DC01CB014D
:104AC000FC01F999FECF06C0F2BDE1BDF89A31961E
:104AD00000B40D9241505040B8F70895DC01CB016D
:104AE00003C02D910E94792541505040D0F7089580
:104AF000262FF999FECF1FBA92BD81BD20BD0FB6FA
:104B0000F894FA9AF99A0FBE019608958F929F929F
:104B1000AF92BF92CF92DF92EF92FF920F931F93CB
:104B2000CF93DF93EC015B016115710519F0FB0177
:104B300091838083F9908F2D90E00E94F426892B39
:104B4000C9F7FDE2FF1621F4F990EE24E39405C0C5
:104B50002BE2F21609F4F990EE248E010150104078
:104B6000C8016CEC70E043E050E00E94FC26892B09
:104B700001F58E010E5F1F4FC8016FEC70E045E03C
:104B800050E00E94FC26892B19F48E01095F1F4F0B
:104B9000A114B10419F0F50111830083E0FC04C0F5
:104BA00070E090E080E814C070E090E080E86FEF83
:104BB00008C1C80164ED70E043E050E00E94FC26AB
:104BC000892B69F4A114B10429F470E090E080EC21
:104BD0006FE7F7C02296F501D183C083F6CF882412
:104BE000992440E050E060E070E0EF2DE053EA30BF
:104BF000A0F5F2E0EF2A8E2D90E09C012870307035
:104C0000E2FE06C0232B79F50894811C911C2BC071
:104C1000232B19F0089481089108DB01CA0112E0E6
:104C2000880F991FAA1FBB1F1A95D1F7480F591F4C
:104C30006A1F7B1F440F551F661F771F4E0F511DA4
:104C4000611D711D483929E9520729E9620729E1E7
:104C5000720748F084E0E82A06C0EE3F31F4E3FC36
:104C600039C098E0E92AF990C0CFE53311F0E53179
:104C700089F529912D3219F4E0E1EE2A05C02B3295
:104C800019F081E090E003C0299182E090E0E22FEA
:104C9000E053EA3018F0C81BD90B1CC020E030E00C
:104CA000FCE020383F075CF4C901880F991F880F8A
:104CB000991F280F391F220F331F2E0F311DE99125
:104CC000E053EA3068F3E4FE03C0309521953F4F8E
:104CD000820E931ECE2CDD24E1FE07C0A114B10488
:104CE00021F02197F501D183C083CB01BA010E9445
:104CF00018277B018C01F3E0CF22DD2423E0C216CC
:104D0000D10421F417FB109517F91095570168018C
:104D1000C801B70120E030E040E050E00E941427D5
:104D2000882309F44AC097FE0DC02BEEE22E20E046
:104D3000F22E9094819491089394C0E2D0E000E028
:104D400010E012C093E0E92E91E0F92EF6CFF701C2
:104D50002591359145915491C601B5010E94442198
:104D60005B016C018C1A9D0A8C169D0684F7D59503
:104D7000C7950F5F1F4F0630110529F08CEF9FEF8D
:104D8000E80EF91EF1CFC501D6017C018D018C2DF5
:104D9000880F8D2D881F8F3F51F0C601B50120E08F
:104DA00030E040E050E00E941427882331F482E292
:104DB00090E09093E0108093DF107E2D9F2D802F48
:104DC000612F272F392F482F562FB901CA01DF91A4
:104DD000CF911F910F91FF90EF90DF90CF90BF90F8
:104DE000AF909F908F900895911183C0803219F0F9
:104DF00089508550D0F70895FB01DC0141505040A7
:104E000088F08D9181341CF08B350CF4805E6591B7
:104E100061341CF06B350CF4605E861B611171F31C
:104E2000990B0895881BFCCF40D008F481E00895C9
:104E3000E89409C097FB3EF4909580957095619534
:104E40007F4F8F4F9F4F9923A9F0F92F96E9BB27EA
:104E50009395F695879577956795B795F111F8CF66
:104E6000FAF4BB0F11F460FF1BC06F5F7F4F8F4FD1
:104E70009F4F16C0882311F096E911C0772321F0C7
:104E80009EE8872F762F05C0662371F096E8862F5F
:104E900070E060E02AF09A95660F771F881FDAF7B6
:104EA000880F9695879597F90895990F0008550FE3
:104EB000AA0BE0E8FEEF16161706E807F907C0F0A0
:104EC00012161306E407F50798F0621B730B840BA8
:104ED000950B39F40A2661F0232B242B252B21F482
:104EE00008950A2609F4A140A6958FEF811D811D22
:0C4EF0000895992788270895F894FFCFB3
:104EFC00526561645F53657475703A20000A0D0049
:104F0C0057726F6E672045454D414749433A200023
:104F1C002F00B400000000000000000000000000A2
:104F2C000000000000000000000000000000000075
:104F3C00000000006400640064006400640064000D
:104F4C006400640009120D0810040B0E0214070112
:104F5C000F050C0009120D0810040B0E02140701AA
:104F6C000F050C000A0A0A0A0A0A0A0A0A0A0A0A9D
:104F7C000A0A0A0A1414141414141414141414140D
:104F8C00141414141E1E1E1E1E1E1E1E1E1E1E1E5D
:104F9C001E1E1E1E646464646464646464646464DD
:104FAC0064646464000102030405060708090A0B23
:104FBC000C0D0E0F0E0F14150C100B191A111612D6
:104FCC000D171318110C1A150F10130B0E180D16B4
:104FDC001719121414120D0F181316110C1A100B9A
:104FEC000E15191716130E140F181510190B0C1A81
:104FFC00120D171115101317120E0C1A0B0F110D91
:10500C00161814190E0F14150C100B191A11161260
:10501C000D17131819110C1A150B140F1810120E5A
:10502C00170D13161613180D170F100B190E12154A
:10503C0014110C1A0E17120F110C1A1510160B1442
:10504C0019130D180B0C0D0E0F101112131415163D
:10505C001718191A000102030405060745525231AC
:10506C000D0A00455252320D0A00455252330D0AB8
:10507C0000455252340D0A0054454D323A20002E50
:10508C00000A0D00505245323A200043414C493A37
:10509C0020003B000305080E1A302E382D31333119
:1050AC0030303632353733000A0D535953494E469A
:1050BC004F3A7A69676269742F72782D70776D3503
:1050CC006334612F61746D656C2F302E382D313344
:1050DC0031303036323537330A0D0053434E003BF6
:1050EC0000200A0D52534900200A0D4C5149002052
:1050FC000A0D41444300200A0D43485600200A0D76
:10510C0046535600200A0D4554433B00200A0D47D8
:10511C00505300200A0D002D2D2D2D2D2D2D2D2D14
:10512C002D2D2D2D2D2D2D2D2D2D2D2D2D2D20528B
:10513C00434F50454E3234202D2D2D2D2D2D2D2D00
:10514C002D2D2D2D2D2D2D2D2D2D2D2D2D2D2D0AA6
:10515C000D00496E666F3A20202020202020202050
:10516C005A696762697420525820354368616E6EC3
:10517C00656C2D536572766F2D50574D0A0D00538B
:10518C00797374656D3A202020202020207A69677D
:10519C006269742F72782D70776D356334612F616D
:1051AC00746D656C2F302E382D31333130303632F2
:1051BC003537330A0D004472697665723A20202027
:1051CC00202020200070776D2D6F757420006E618B
:1051DC007574696328004368616E6E656C732D3E4F
:1051EC00536572766F2D003B200078007573292073
:1051FC000074656C656D6574726965200066616923
:10520C006C73617665200020202020202020202037
:10521C002020202020200A0D0050726F746F636FC5
:10522C006C2020202020200064737373200066689B
:10523C00737320007468737320006C697374656EEB
:10524C002D6265666F72652D74616C6B2000525314
:10525C0053492864426D293A20202020002C00203C
:10526C0020202020202020202020202020200A0D5B
:10527C004E4F4953452864426D293A202020002086
:10528C0020202020202020202020202020200A0D3B
:10529C00534E2D44696666286442293A202000202A
:1052AC0020202020202020202020202020200A0D1B
:1052BC004C51493A20202020202020202020002062
:1052CC0020202020202020202020202020200A0DFB
:1052DC004552524F52533A202020202020200028A3
:1052EC00002F0020002529202020202020202020F5
:1052FC002020202020200A0D484F50503A202020FA
:10530C0020202020202000202020202020202020B1
:10531C0020202020202020200A0D547849443A20B7
:10532C0020202020202020200020280029202020A0
:10533C002020202020202020202020200A0D534532
:10534C00513A202020202020202020200020202026
:10535C002020202020202020200A0D00414443271B
:10536C00733A2020202020202020303D0020313D89
:10537C000020323D0020333D00202020200A0D006B
:10538C004F534343414C202020202020202000203C
:10539C002020202020200A0D005461626C65733A95
:1053AC0020202020202020002C200056616C7565C8
:1053BC00732020202020202020004C6173742D4D60
:1053CC00756C74694E756D20004D756C74697661E1
:1053DC006C756573202020002D3E002920002020B4
:1053EC0020202020200A0D4D756C746976616C7537
:1053FC006573322020004D543A003A0020200A0DEB
:10540C00002D2D2D2D2D2D2D2D2D2D2D2D2D2D2DED
:10541C002D2D2D2D2D2D0A0D003E003D004D453A14
:10542C00000A0D0072636F70656E32342D72782035
:10543C00285A696762697420525820354368616E36
:10544C006E656C2D536572766F2D50574D290A0D74
:10545C000053657474696E672046616C6573617680
:10546C00652D56616C7565730A0D00536574757006
:10547C002D53617665640A0D004D756C74697072FC
:10548C006F702D53657474696E67730A0D002E2E40
:10549C002E73617665642E2E2E002E2E2E72657361
:1054AC0065742E2E2E0062696E642E2E2E2E0A0D21
:1054BC0000010303030300000000000000000303CD
:1054CC000303030303030404040404040404040496
:1054DC000404040404040404040404040404020284
:1054EC000302020303030302030303030203030384
:1054FC0003032B0E2F0E300E310E320E330E350EE3
:10550C00370E390E3B0E3D0E3F0E410E430E440E30
:10551C00450E460E470E480E490E4A0E4B0E4C0ECB
:10552C004D0E4E0E4F0E500E510E520E530E540E7B
:10553C00550E560E570E580E590E5A0E5B0E5C0E2B
:10554C005D0E5E0E5F0E600E610E620E630E650EDA
:10555C00670E680E6A0E6C0E6D0E6E0E6F0E700E70
:10556C00720E730E740E750E760E780E790E7A0E10
:10557C007B0E7C0E6964007461626C650074696DED
:10558C00657461626C65004661696C736176654D2A
:10559C006F6465004661696C736176655365740070
:1055AC004661696C7361766556616C7565735F31C4
:1055BC00004661696C7361766556616C7565735FE5
:1055CC0032004661696C7361766556616C75657302
:1055DC005F33004661696C7361766556616C756505
:1055EC00735F34004661696C7361766556616C75E6
:1055FC0065735F35004661696C7361766556616CE5
:10560C007565735F36004661696C736176655661CA
:10561C006C7565735F37004661696C7361766556AE
:10562C00616C7565735F3800536572766F4D617090
:10563C005F3100536572766F4D61705F3200536558
:10564C0072766F4D61705F3300536572766F4D618A
:10565C00705F3400536572766F4D61705F35005327
:10566C006572766F4D61705F3600536572766F4D63
:10567C0061705F3700536572766F4D61705F3800F3
:10568C00536572766F4475616C526174655F31005D
:10569C00536572766F4475616C526174655F32004C
:1056AC00536572766F4475616C526174655F33003B
:1056BC00536572766F4475616C526174655F34002A
:1056CC00536572766F4475616C526174655F350019
:1056DC00536572766F4475616C526174655F360008
:1056EC00536572766F4475616C526174655F3700F7
:1056FC00536572766F4475616C526174655F3800E6
:10570C00536572766F41747655705F3100536572D4
:10571C00766F41747655705F3200536572766F41C7
:10572C00747655705F3300536572766F417476559D
:10573C00705F3400536572766F41747655705F35C7
:10574C0000536572766F41747655705F3600536501
:10575C0072766F41747655705F3700536572766F51
:10576C0041747655705F3800536572766F4174766C
:10577C00446F776E5F3100536572766F4174764477
:10578C006F776E5F3200536572766F417476446F3B
:10579C00776E5F3300536572766F417476446F7722
:1057AC006E5F3400536572766F417476446F776E1A
:1057BC005F3500536572766F417476446F776E5F18
:1057CC003600536572766F417476446F776E5F372F
:1057DC0000536572766F417476446F776E5F380054
:1057EC0050574D526174655F310050574D52617482
:1057FC00655F320050504D4368616E6E656C73008E
:10580C0050504D53796E630050504D536869667417
:10581C000050504D496E76657274006D756C7469EC
:10582C005F6368616E6E656C006D756C74695F6347
:10583C0068616E6E656C73006D756C74695F6D7309
:10584C00796E635F6E756D006D756C74695F6D73E9
:10585C00796E635F6C656E006D756C74695F6368FF
:10586C00616E6E656C6D6170006D756C7469325F24
:10587C006368616E6E656C006D756C7469325F6324
:10588C0068616E6E656C73006D756C7469325F6DFA
:10589C0073796E635F6E756D006D756C7469325FD4
:1058AC006D73796E635F6C656E006D756C746932C7
:1058BC005F6368616E6E656C6D6170006D656E75B1
:1058CC005F6C656E006373765F6F757470757400D2
:1058DC0073617665006D756C74697365740084080A
:1058EC0087088D089708A408B008C108D208E308F7
:1058FC00F408050916092709380943094E095909FD
:10590C0064096F097A0985099009A009B009C009D1
:10591C00D009E009F009000A100A1D0A2A0A370A00
:10592C00440A510A5E0A6B0A780A870A960AA50A83
:10593C00B40AC30AD20AE10AF00AFA0A040B100BE1
:10594C00180B210B2B0B390B480B580B680B790BD5
:10595C00880B980BA90BBA0BCC0BD50BE00BE50BFA
:10596C00476C6F62616C004661696C7361766500AF
:10597C00536572766F2D4D6170004475616C726168
:10598C007465004174762D5570004174762D446F0A
:10599C00776E0050574D2D4F7574707574005050C4
:1059AC004D2D4F7574707574004D756C74697072F3
:1059BC006F70004D756C746970726F7032004D654C
:1059CC006E7500700C770C800C8A0C930C9A0CA3DF
:1059DC000CAE0CB90CC30CCE0C00030D151D252DF3
:1059EC002F33383D030A0808080802040505040192
:1059FC00010101010101010101010101010101018B
:105A0C00010101010101010101010101010101FF7C
:0A5A1C00010000000000000000007F
:00000001FF
